
C:\Documents and Settings\jarek\Pulpit\Privet\Magisterka\Programy\1\um0427\FWLib\project\RIDE\STM3210E-EVAL\BUZER.o:     file format elf32-littlearm
C:\Documents and Settings\jarek\Pulpit\Privet\Magisterka\Programy\1\um0427\FWLib\project\RIDE\STM3210E-EVAL\BUZER.o

Disassembly of section .text.BUZER_Beep:

00000000 <BUZER_Beep>:
BUZER_Beep():
C:\Documents and Settings\jarek\Pulpit\Privet\Magisterka\Programy\1\um0427\FWLib\project/BUZER.c:43
   0:	4a02      	ldr	r2, [pc, #8]	(c <BUZER_Beep+0xc>)
   2:	2301      	movs	r3, #1
   4:	7013      	strb	r3, [r2, #0]
C:\Documents and Settings\jarek\Pulpit\Privet\Magisterka\Programy\1\um0427\FWLib\project/BUZER.c:44
   6:	6050      	str	r0, [r2, #4]
C:\Documents and Settings\jarek\Pulpit\Privet\Magisterka\Programy\1\um0427\FWLib\project/BUZER.c:45
   8:	4770      	bx	lr
   a:	46c0      	nop			(mov r8, r8)
   c:	00000000 	.word	0x00000000
Disassembly of section .text.BUZER_Song:

00000000 <BUZER_Song>:
BUZER_Song():
C:\Documents and Settings\jarek\Pulpit\Privet\Magisterka\Programy\1\um0427\FWLib\project/BUZER.c:48
   0:	4b01      	ldr	r3, [pc, #4]	(8 <BUZER_Song+0x8>)
   2:	2203      	movs	r2, #3
   4:	701a      	strb	r2, [r3, #0]
C:\Documents and Settings\jarek\Pulpit\Privet\Magisterka\Programy\1\um0427\FWLib\project/BUZER.c:49
   6:	4770      	bx	lr
   8:	00000000 	.word	0x00000000
Disassembly of section .text.BUZER_OnOff:

00000000 <BUZER_OnOff>:
BUZER_OnOff():
C:\Documents and Settings\jarek\Pulpit\Privet\Magisterka\Programy\1\um0427\FWLib\project/BUZER.c:33
   0:	b510      	push	{r4, lr}
C:\Documents and Settings\jarek\Pulpit\Privet\Magisterka\Programy\1\um0427\FWLib\project/BUZER.c:34
   2:	b120      	cbz	r0, e <BUZER_OnOff+0xe>
C:\Documents and Settings\jarek\Pulpit\Privet\Magisterka\Programy\1\um0427\FWLib\project/BUZER.c:35
   4:	4804      	ldr	r0, [pc, #16]	(18 <BUZER_OnOff+0x18>)
   6:	2110      	movs	r1, #16
   8:	f7ff fffe 	bl	0 <GPIO_SetBits>
   c:	e003      	b.n	16 <BUZER_OnOff+0x16>
C:\Documents and Settings\jarek\Pulpit\Privet\Magisterka\Programy\1\um0427\FWLib\project/BUZER.c:37
   e:	4802      	ldr	r0, [pc, #8]	(18 <BUZER_OnOff+0x18>)
  10:	2110      	movs	r1, #16
  12:	f7ff fffe 	bl	0 <GPIO_ResetBits>
C:\Documents and Settings\jarek\Pulpit\Privet\Magisterka\Programy\1\um0427\FWLib\project/BUZER.c:39
  16:	bd10      	pop	{r4, pc}
  18:	0800      	.short	0x0800
  1a:	4001      	.short	0x4001
Disassembly of section .text.BUZER_Thret:

00000000 <BUZER_Thret>:
BUZER_Thret():
C:\Documents and Settings\jarek\Pulpit\Privet\Magisterka\Programy\1\um0427\FWLib\project/BUZER.c:52
   0:	4b31      	ldr	r3, [pc, #196]	(c8 <BUZER_Thret+0xc8>)
C:\Documents and Settings\jarek\Pulpit\Privet\Magisterka\Programy\1\um0427\FWLib\project/BUZER.c:51
   2:	b510      	push	{r4, lr}
C:\Documents and Settings\jarek\Pulpit\Privet\Magisterka\Programy\1\um0427\FWLib\project/BUZER.c:52
   4:	781b      	ldrb	r3, [r3, #0]
   6:	3b01      	subs	r3, #1
   8:	2b08      	cmp	r3, #8
   a:	d85c      	bhi.n	c6 <BUZER_Thret+0xc6>
   c:	e8df f003 	tbb	[pc, r3]
  10:	1a130905 	.word	0x1a130905
  14:	40382d25 	.word	0x40382d25
  18:	0052      	.short	0x0052
C:\Documents and Settings\jarek\Pulpit\Privet\Magisterka\Programy\1\um0427\FWLib\project/BUZER.c:56
  1a:	4b2b      	ldr	r3, [pc, #172]	(c8 <BUZER_Thret+0xc8>)
  1c:	2202      	movs	r2, #2
  1e:	701a      	strb	r2, [r3, #0]
C:\Documents and Settings\jarek\Pulpit\Privet\Magisterka\Programy\1\um0427\FWLib\project/BUZER.c:57
  20:	e051      	b.n	c6 <BUZER_Thret+0xc6>
C:\Documents and Settings\jarek\Pulpit\Privet\Magisterka\Programy\1\um0427\FWLib\project/BUZER.c:59
  22:	4c29      	ldr	r4, [pc, #164]	(c8 <BUZER_Thret+0xc8>)
  24:	6863      	ldr	r3, [r4, #4]
  26:	2b00      	cmp	r3, #0
  28:	dc36      	bgt.n	98 <BUZER_Thret+0x98>
C:\Documents and Settings\jarek\Pulpit\Privet\Magisterka\Programy\1\um0427\FWLib\project/BUZER.c:63
  2a:	2000      	movs	r0, #0
  2c:	f7ff fffe 	bl	0 <BUZER_Thret>
C:\Documents and Settings\jarek\Pulpit\Privet\Magisterka\Programy\1\um0427\FWLib\project/BUZER.c:64
  30:	2300      	movs	r3, #0
  32:	7023      	strb	r3, [r4, #0]
  34:	e047      	b.n	c6 <BUZER_Thret+0xc6>
C:\Documents and Settings\jarek\Pulpit\Privet\Magisterka\Programy\1\um0427\FWLib\project/BUZER.c:68
  36:	4b24      	ldr	r3, [pc, #144]	(c8 <BUZER_Thret+0xc8>)
  38:	2204      	movs	r2, #4
  3a:	701a      	strb	r2, [r3, #0]
C:\Documents and Settings\jarek\Pulpit\Privet\Magisterka\Programy\1\um0427\FWLib\project/BUZER.c:69
  3c:	f502 72c6 	add.w	r2, r2, #396	; 0x18c
  40:	605a      	str	r2, [r3, #4]
C:\Documents and Settings\jarek\Pulpit\Privet\Magisterka\Programy\1\um0427\FWLib\project/BUZER.c:70
  42:	e040      	b.n	c6 <BUZER_Thret+0xc6>
C:\Documents and Settings\jarek\Pulpit\Privet\Magisterka\Programy\1\um0427\FWLib\project/BUZER.c:72
  44:	4c20      	ldr	r4, [pc, #128]	(c8 <BUZER_Thret+0xc8>)
  46:	6863      	ldr	r3, [r4, #4]
  48:	2b00      	cmp	r3, #0
  4a:	dc25      	bgt.n	98 <BUZER_Thret+0x98>
C:\Documents and Settings\jarek\Pulpit\Privet\Magisterka\Programy\1\um0427\FWLib\project/BUZER.c:76
  4c:	2000      	movs	r0, #0
  4e:	f7ff fffe 	bl	0 <BUZER_Thret>
C:\Documents and Settings\jarek\Pulpit\Privet\Magisterka\Programy\1\um0427\FWLib\project/BUZER.c:77
  52:	2305      	movs	r3, #5
  54:	7023      	strb	r3, [r4, #0]
C:\Documents and Settings\jarek\Pulpit\Privet\Magisterka\Programy\1\um0427\FWLib\project/BUZER.c:78
  56:	33c3      	adds	r3, #195
  58:	e02a      	b.n	b0 <BUZER_Thret+0xb0>
C:\Documents and Settings\jarek\Pulpit\Privet\Magisterka\Programy\1\um0427\FWLib\project/BUZER.c:82
  5a:	4a1b      	ldr	r2, [pc, #108]	(c8 <BUZER_Thret+0xc8>)
  5c:	6853      	ldr	r3, [r2, #4]
  5e:	2b00      	cmp	r3, #0
  60:	dc2c      	bgt.n	bc <BUZER_Thret+0xbc>
C:\Documents and Settings\jarek\Pulpit\Privet\Magisterka\Programy\1\um0427\FWLib\project/BUZER.c:85
  62:	2306      	movs	r3, #6
  64:	7013      	strb	r3, [r2, #0]
C:\Documents and Settings\jarek\Pulpit\Privet\Magisterka\Programy\1\um0427\FWLib\project/BUZER.c:86
  66:	33c2      	adds	r3, #194
  68:	e029      	b.n	be <BUZER_Thret+0xbe>
C:\Documents and Settings\jarek\Pulpit\Privet\Magisterka\Programy\1\um0427\FWLib\project/BUZER.c:90
  6a:	4c17      	ldr	r4, [pc, #92]	(c8 <BUZER_Thret+0xc8>)
  6c:	6863      	ldr	r3, [r4, #4]
  6e:	2b00      	cmp	r3, #0
  70:	dc12      	bgt.n	98 <BUZER_Thret+0x98>
C:\Documents and Settings\jarek\Pulpit\Privet\Magisterka\Programy\1\um0427\FWLib\project/BUZER.c:94
  72:	2000      	movs	r0, #0
  74:	f7ff fffe 	bl	0 <BUZER_Thret>
C:\Documents and Settings\jarek\Pulpit\Privet\Magisterka\Programy\1\um0427\FWLib\project/BUZER.c:95
  78:	2307      	movs	r3, #7
  7a:	7023      	strb	r3, [r4, #0]
C:\Documents and Settings\jarek\Pulpit\Privet\Magisterka\Programy\1\um0427\FWLib\project/BUZER.c:96
  7c:	33c1      	adds	r3, #193
  7e:	e017      	b.n	b0 <BUZER_Thret+0xb0>
C:\Documents and Settings\jarek\Pulpit\Privet\Magisterka\Programy\1\um0427\FWLib\project/BUZER.c:100
  80:	4a11      	ldr	r2, [pc, #68]	(c8 <BUZER_Thret+0xc8>)
  82:	6853      	ldr	r3, [r2, #4]
  84:	2b00      	cmp	r3, #0
  86:	dc19      	bgt.n	bc <BUZER_Thret+0xbc>
C:\Documents and Settings\jarek\Pulpit\Privet\Magisterka\Programy\1\um0427\FWLib\project/BUZER.c:103
  88:	2308      	movs	r3, #8
  8a:	7013      	strb	r3, [r2, #0]
C:\Documents and Settings\jarek\Pulpit\Privet\Magisterka\Programy\1\um0427\FWLib\project/BUZER.c:104
  8c:	33c0      	adds	r3, #192
  8e:	e016      	b.n	be <BUZER_Thret+0xbe>
C:\Documents and Settings\jarek\Pulpit\Privet\Magisterka\Programy\1\um0427\FWLib\project/BUZER.c:108
  90:	4c0d      	ldr	r4, [pc, #52]	(c8 <BUZER_Thret+0xc8>)
  92:	6863      	ldr	r3, [r4, #4]
  94:	2b00      	cmp	r3, #0
  96:	dd05      	ble.n	a4 <BUZER_Thret+0xa4>
C:\Documents and Settings\jarek\Pulpit\Privet\Magisterka\Programy\1\um0427\FWLib\project/BUZER.c:109
  98:	3b01      	subs	r3, #1
C:\Documents and Settings\jarek\Pulpit\Privet\Magisterka\Programy\1\um0427\FWLib\project/BUZER.c:110
  9a:	2001      	movs	r0, #1
C:\Documents and Settings\jarek\Pulpit\Privet\Magisterka\Programy\1\um0427\FWLib\project/BUZER.c:109
  9c:	6063      	str	r3, [r4, #4]
C:\Documents and Settings\jarek\Pulpit\Privet\Magisterka\Programy\1\um0427\FWLib\project/BUZER.c:110
  9e:	f7ff fffe 	bl	0 <BUZER_Thret>
  a2:	e010      	b.n	c6 <BUZER_Thret+0xc6>
C:\Documents and Settings\jarek\Pulpit\Privet\Magisterka\Programy\1\um0427\FWLib\project/BUZER.c:112
  a4:	2000      	movs	r0, #0
  a6:	f7ff fffe 	bl	0 <BUZER_Thret>
C:\Documents and Settings\jarek\Pulpit\Privet\Magisterka\Programy\1\um0427\FWLib\project/BUZER.c:113
  aa:	2309      	movs	r3, #9
  ac:	7023      	strb	r3, [r4, #0]
C:\Documents and Settings\jarek\Pulpit\Privet\Magisterka\Programy\1\um0427\FWLib\project/BUZER.c:114
  ae:	33bf      	adds	r3, #191
  b0:	6063      	str	r3, [r4, #4]
  b2:	e008      	b.n	c6 <BUZER_Thret+0xc6>
C:\Documents and Settings\jarek\Pulpit\Privet\Magisterka\Programy\1\um0427\FWLib\project/BUZER.c:118
  b4:	4a04      	ldr	r2, [pc, #16]	(c8 <BUZER_Thret+0xc8>)
  b6:	6853      	ldr	r3, [r2, #4]
  b8:	2b00      	cmp	r3, #0
  ba:	dd02      	ble.n	c2 <BUZER_Thret+0xc2>
C:\Documents and Settings\jarek\Pulpit\Privet\Magisterka\Programy\1\um0427\FWLib\project/BUZER.c:119
  bc:	3b01      	subs	r3, #1
  be:	6053      	str	r3, [r2, #4]
  c0:	e001      	b.n	c6 <BUZER_Thret+0xc6>
C:\Documents and Settings\jarek\Pulpit\Privet\Magisterka\Programy\1\um0427\FWLib\project/BUZER.c:121
  c2:	2300      	movs	r3, #0
  c4:	7013      	strb	r3, [r2, #0]
C:\Documents and Settings\jarek\Pulpit\Privet\Magisterka\Programy\1\um0427\FWLib\project/BUZER.c:125
  c6:	bd10      	pop	{r4, pc}
  c8:	00000000 	.word	0x00000000
Disassembly of section .text.BUZER_Init:

00000000 <BUZER_Init>:
BUZER_Init():
C:\Documents and Settings\jarek\Pulpit\Privet\Magisterka\Programy\1\um0427\FWLib\project/BUZER.c:24
   0:	b507      	push	{r0, r1, r2, lr}
C:\Documents and Settings\jarek\Pulpit\Privet\Magisterka\Programy\1\um0427\FWLib\project/BUZER.c:28
   2:	2302      	movs	r3, #2
C:\Documents and Settings\jarek\Pulpit\Privet\Magisterka\Programy\1\um0427\FWLib\project/BUZER.c:27
   4:	2210      	movs	r2, #16
C:\Documents and Settings\jarek\Pulpit\Privet\Magisterka\Programy\1\um0427\FWLib\project/BUZER.c:30
   6:	4805      	ldr	r0, [pc, #20]	(1c <BUZER_Init+0x1c>)
   8:	a901      	add	r1, sp, #4
C:\Documents and Settings\jarek\Pulpit\Privet\Magisterka\Programy\1\um0427\FWLib\project/BUZER.c:27
   a:	f8ad 2004 	strh.w	r2, [sp, #4]
C:\Documents and Settings\jarek\Pulpit\Privet\Magisterka\Programy\1\um0427\FWLib\project/BUZER.c:28
   e:	f88d 3006 	strb.w	r3, [sp, #6]
C:\Documents and Settings\jarek\Pulpit\Privet\Magisterka\Programy\1\um0427\FWLib\project/BUZER.c:29
  12:	f88d 2007 	strb.w	r2, [sp, #7]
C:\Documents and Settings\jarek\Pulpit\Privet\Magisterka\Programy\1\um0427\FWLib\project/BUZER.c:30
  16:	f7ff fffe 	bl	0 <GPIO_Init>
C:\Documents and Settings\jarek\Pulpit\Privet\Magisterka\Programy\1\um0427\FWLib\project/BUZER.c:31
  1a:	bd0e      	pop	{r1, r2, r3, pc}
  1c:	40010800 	.word	0x40010800
